:100000000C9458060C9480060C9480060C94800680
:100010000C9480060C9480060C94ED180C948006C9
:100020000C9480060C9480060C9480060C94800638
:100030000C9480060C9480060C9480060C94800628
:100040000C94A3180C9480060C9471180C944B1803
:100050000C9480060C9480060C9480060C94800608
:100060000C9404190C9480061FC01FC03FC03F8031
:100070007F007FC0FFC0FF801F003E003C00780073
:10008000700060001FC0104020402080410043C02D
:100090008040F080110022002400480050006000E1
:1000A00000000000003E5B4F5B3E3E6B4F6B3E1C12
:1000B0003E7C3E1C183C7E3C181C577D571C1C5E29
:1000C0007F5E1C00183C1800FFE7C3E7FF00182400
:1000D0001800FFE7DBE7FF30483A060E26297929AA
:1000E00026407F050507407F05253F5A3CE73C5ADF
:1000F0007F3E1C1C08081C1C3E7F14227F22145FBC
:100100005F005F5F06097F017F006689956A606016
:1001100060606094A2FFA29408047E040810207E10
:10012000201008082A1C08081C2A08081E10101095
:10013000100C1E0C1E0C30383E3830060E3E0E06DB
:10014000000000000000005F00000007000700142E
:100150007F147F14242A7F2A1223130864623649ED
:100160005620500008070300001C224100004122D5
:100170001C002A1C7F1C2A08083E080800807030DA
:100180000008080808080000606000201008040249
:100190003E5149453E00427F40007249494946214F
:1001A00041494D331814127F1027454545393C4AC3
:1001B00049493141211109073649494936464949DA
:1001C000291E000014000000403400000008142222
:1001D0004114141414140041221408020159090690
:1001E0003E415D594E7C1211127C7F494949363E91
:1001F000414141227F4141413E7F494949417F0977
:100200000909013E414151737F0808087F00417F81
:1002100041002040413F017F081422417F4040407F
:10022000407F021C027F7F0408107F3E4141413E17
:100230007F090909063E4151215E7F091929462699
:100240004949493203017F01033F4040403F1F209D
:1002500040201F3F4038403F631408146303047874
:1002600004036159494D43007F4141410204081094
:1002700020004141417F04020102044040404040CF
:10028000000307080020545478407F28444438383D
:1002900044444428384444287F38545454180008AF
:1002A0007E090218A4A49C787F0804047800447D89
:1002B00040002040403D007F1028440000417F4026
:1002C000007C047804787C0804047838444444387A
:1002D000FC1824241818242418FC7C08040408485A
:1002E0005454542404043F44243C4040207C1C20AB
:1002F00040201C3C4030403C44281028444C909006
:10030000907C4464544C440008364100000077005F
:1003100000004136080002010204023C2623263C6C
:100320001EA1A161123A4040207A385454555921F7
:1003300055557941225454784221555478402054DF
:100340005579400C1E52721239555555593954542D
:10035000545939555454580000457C410002457D9C
:10036000420001457C407D1211127DF0282528F0C5
:100370007C545545002054547C547C0A097F4932F2
:10038000494949323A4444443A324A4848303A4169
:1003900041217A3A42402078009DA0A07D3D424212
:1003A000423D3D4040403D3C24FF2424487E49439B
:1003B000662B2FFC2F2BFF0929F620C0887E09030E
:1003C00020545479410000447D413048484A323835
:1003D0004040227A007A0A0A727D0D19317D262961
:1003E000292F28262929292630484D402038080859
:1003F000080808080808382F10C8ACBA2F1028348D
:10040000FA00007B000008142A142222142A14087F
:100410005500550055AA55AA55AAFF55FF55FF008E
:100420000000FF00101010FF00141414FF00101043
:10043000FF00FF1010F010F0141414FC001414F757
:1004400000FF0000FF00FF1414F404FC1414171044
:100450001F10101F101F1414141F00101010F00094
:100460000000001F101010101F10101010F01000CE
:100470000000FF101010101010101010FF100000DE
:1004800000FF140000FF00FF00001F10170000FC19
:1004900004F414141710171414F404F40000FF00EB
:1004A000F714141414141414F700F7141414171474
:1004B00010101F101F141414F4141010F010F0007A
:1004C000001F101F0000001F14000000FC1400009B
:1004D000F010F01010FF10FF141414FF141010107F
:1004E0001F00000000F010FFFFFFFFFFF0F0F0F032
:1004F000F0FFFFFF0000000000FFFF0F0F0F0F0FC6
:100500003844443844FC4A4A4A347E020206060211
:100510007E027E0263554941633844443C04407E78
:10052000201E2006027E020299A5E7A5991C2A49F1
:100530002A1C4C7201724C304A4D4D30304878487C
:1005400030BC625A463D3E494949007E0101017E68
:100550002A2A2A2A2A44445F444440514A444040BB
:10056000444A51400000FF0103E080FF00000808FA
:100570006B6B083612362436060F090F060000187A
:10058000180000001010003040FF0101001F0101A1
:100590001E00191D1712003C3C3C3C0000000000EE
:1005A000000103070F1F3F7F0080C0E0F0F8FCFE52
:1005B00000000000230026002900000000080002BF
:1005C000010000030407000000000000000000001C
:1005D0000000240027002A00DB40A4A62EAFDA0288
:1005E00081DA1281DA02818F2000A1C8D300408D08
:1005F000AED580A801020408102040800102040842
:10060000102001020408102000000000250028002E
:100610002B00040404040404040402020202020283
:100620000303030303030000600000000000000058
:1006300000000000000000E00000000000000000DA
:10064000000000000001E0000000000000000000C9
:100650000000000001F000000000000000000000A9
:1006600000000003F0000000000000000000000097
:10067000000007F000000000000000000000000083
:100680000007F8000000000000000000000000006B
:100690000FF800000003C0007E000001E0007F0FA3
:1006A000F800000003C000FE000001E000FFEFF8CA
:1006B00000000003C000FE000001E000FFFFF800A2
:1006C000000003C000F00000000F007FFE7FC000AC
:1006D0000003C000F00000000F003FFE7FF83FF174
:1006E000FBCFFCFEF3BC3DEFE01FFE7FFF7FFBFF77
:1006F000DFFEFEFFBC3DEFE01FC6FFFF7FFBFFDF1D
:10070000FEFEFFBC3DEFE00FE3C7FE787BC3DE1EBD
:10071000F0FFBC3DEF0007FF87FC787BC3DE1EF0D7
:10072000F83C3DEF0001FFFFF0007BC3C01EF0F07E
:100730003C3DEF0001F37FE03FFBC3CFFEF0F03C18
:100740003DEF0003E33F807FFBC3DFFEF0F03C3D65
:10075000EF0007E73C00787BC3DE1EF0F03C3DEF86
:100760000007FFBE00787BC3DE1EF0F03C3DEF00CB
:1007700007FFFE00787BC3DE1EF0F03C3DEF000F6C
:10078000FFFE007FFBFFDFFEF0F03FFDEFE00FFF1D
:10079000FF007FFBFFDFFEF0F03FFDEFE00FF9FF12
:1007A000003E79F9CF9EF0F01F3DE7E01FF1FF001A
:1007B00000000000000000000000001F80FF007F1C
:1007C000FFFFFFFFFFFFFFFFFFE01C007F007FFF39
:1007D000FFFFFEB46D888D18E000001F007FFFFF53
:1007E000FFFE95AD7DB577E000000F007FFFFFFFB6
:1007F000FEA5AD9D8D19E0000006007FFFFFFFFE06
:10080000B5ADEDB57EE00000000000018000000005
:100810000000000000000380000000000000000055
:100820000007C000000000000000000007C000003A
:10083000000000000000000FC000000000000000E9
:1008400000001FE00000000000000000001FE000AA
:1008500000000000000000003FE000000000000079
:100860000000003FF00000000000000000007FF0EA
:10087000000000000000001FF87FF00000000000F2
:1008800000003FFE7FF0000000000000003FFF7FFF
:10089000F0000000000000001FFFFBE0000000006F
:1008A0000000000FFFF9FFC00000000000000FFF74
:1008B000F9FFF800000000000007FFF1FFFF000053
:1008C0000000000003FC73FFFF8000000000000137
:1008D000FE3FFFFF80000000000000FF1E0FFF0032
:1008E0000000000000007FFE1FFC00000000000070
:1008F000003FFFFFF8000000000000000FDFFFE0F6
:10090000000000000000001F19FFC00000000000F0
:1009100000003F3CFF00000000000000007E7CF86B
:1009200000000000000000007FFE7C0000000000CE
:10093000000000FFFFFC0000000000000000FFFFBF
:10094000FE0000000000000000FFFFFE00000000AD
:1009500000000001FFEFFE0000000000000001FFAA
:10096000CFFE0000000000000003FF07FE000000B3
:100970000000000003FC07FE000000000000000370
:10098000F003FE00000000000000018000FE0000F7
:1009900000000000000000007E00000000000000D9
:1009A0000000003E000000000000000000000C00FD
:1009B0000000000000078000FC000003C0000000F1
:1009C000078001FC000003C0000000078001FC005C
:1009D0000003C0000000078001E00000001E0000CE
:1009E00000078001E00000001E007FE3F79FF9FD93
:1009F000E7787BDFC0FFF7FFBFFDFDFF787BDFC03F
:100A0000FFF7FFBFFDFDFF787BDFC0F0F787BC3D40
:100A1000E1FF787BDE00F0F787BC3DE1F0787BDE1C
:100A20000000F787803DE1E0787BDE007FF7879F5D
:100A3000FDE1E0787BDE00FFF787BFFDE1E0787B3A
:100A4000DE00F0F787BC3DE1E0787BDE00F0F78761
:100A5000BC3DE1E0787BDE00F0F787BC3DE1E0786B
:100A60007BDE00FFF7FFBFFDE1E07FFBDFC0FFF7AC
:100A7000FFBFFDE1E07FFBDFC07CF3F39F3DE1E0E2
:100A80003E7BCFC00000000000000000000000FF1F
:100A9000FFFFFFFFFFFFFFFFFFC0FFFFFFFFFD683E
:100AA000DB111A31C0FFFFFFFFFD2B5AFB6AEFC0BD
:100AB000FFFFFFFFFD4B5B3B1A33C0FFFFFFFFFD56
:100AC0006B5BDB6AFDC003FFFFFFFFFFFFFFFFFF64
:100AD000FFFFFFC0000FFFFFFFFFFFFFFFFFFFFF54
:100AE000FFFFF0001FFFFFFFFFFFFFFFFFFFFFFF04
:100AF000FFF8003FFFFFFFFFFFFFFFFFFFFFFFFFCC
:100B0000FC007FFFFFFFFFFFFFFFFFFFFFFFFFFE78
:100B1000007FFFFFFFFFFFFFFFFFFFFFFFFFFE0064
:100B2000FFFFFFFFFFFFFFFFFFFFFFFFFFFF00FFD4
:100B3000FFFFFFFFFFFFFFFFFFFFFFFFFF00FFFFC4
:100B4000FFFFFFFFFFFFFFFFFFFFFFFF00FFFFFFB4
:100B5000FFFFFFFFFFFFFFFFFFFFFF00FFFFFFFFA4
:100B6000FFFFFFFFFFFFFFFFFFFF00FFFFFFFFFF94
:100B7000FFFFFFFFFFFFFFFFFF60FFFFFFFFFFFF24
:100B8000FFFFFFFFFFFFFFFF70FFFFFFFFFFFFFF04
:100B9000FFFFFFFFFFFFFF78FFFFFFFFFFFFFFFFEC
:100BA000FFFFFFFFFFFF78FFFFFFFFFFFFFFFFFFDC
:100BB000FFFFFFFFFF78FFFFFFFFFFFFFFFFFFFFCC
:100BC000FFFFFFFF78FFFFFFFFFFFFFFFFFFFFFFBC
:100BD000FFFFFF78FFFFFFFFFFFFFFFFFFFFFFFFAC
:100BE000FFFF78FFFFFFFFFFFFFFFFFFFFFFFFFF9C
:100BF000FF70FFFFFFFFFFFFFFFFFFFFFFFFFFFF94
:100C000060FFFFFFFFFFFFFFFFFFFFFFFFFFFF0092
:100C1000FFFFFFFFFFFFFFFFFFFFFFFFFFFF00FFE3
:100C2000FFFFFFFFFFFFFFFFFFFFFFFFFF00FFFFD3
:100C3000FFFFFFFFFFFFFFFFFFFFFFFF00FFFFFFC3
:100C4000FFFFFFFFFFFFFFFFFFFFFF007FFFFFFF33
:100C5000FFFFFFFFFFFFFFFFFFFE007FFFFFFFFF24
:100C6000FFFFFFFFFFFFFFFFFE003FFFFFFFFFFF54
:100C7000FFFFFFFFFFFFFFFC001FFFFFFFFFFFFF66
:100C8000FFFFFFFFFFFFF8000FFFFFFFFFFFFFFF6A
:100C9000FFFFFFFFFFF00003FFFFFFFFFFFFFFFF6E
:100CA000FFFFFFFFC0002200FF210000231AC31F27
:100CB00011241FBECFEFD8E0DEBFCDBF13E0A0E010
:100CC000B1E0E6EFF6E402C005900D92A039B1075D
:100CD000D9F725E0A0E9B3E001C01D92A534B20721
:100CE000E1F716E0C7E5D6E004C02197FE010E94B7
:100CF0003722C635D107C9F70E94B21A0C946E2369
:100D00000C940000982F2091540481E0213208F0C7
:100D100043C0809130048111FCCF8091530432E0B4
:100D20003093300490932F049FEF90932E041092F1
:100D30002D0420932C04A3E3B4E0ECE0F4E090E075
:100D4000291331C010920B0490910B04880F892B4A
:100D500080930B0480910A04813049F510920A04B3
:100D600080910B048093BB008091BC0083FDF8CF81
:100D700085EC8093BC00809130048230E1F3809157
:100D80002E048F3FB1F080912E048032A1F080912B
:100D90002E04803391F084E01092320410925404B7
:100DA0001092310408953D9131939F5FC9CF85EE34
:100DB000E0CF80E0F1CF82E0EFCF83E0EDCF089588
:100DC00008950895AF92BF92CF92DF92EF92FF9273
:100DD0000F931F93CF93DF936C017B018B01040F63
:100DE000151FEB015E01AE18BF08C017D10759F0FF
:100DF0006991D601ED91FC910190F081E02DC60141
:100E00000995892B79F7C501DF91CF911F910F913A
:100E1000FF90EF90DF90CF90BF90AF900895FC01CE
:100E2000538D448D252F30E0842F90E0821B930B4F
:100E3000541710F0CF96089501970895FC01918DF5
:100E4000828D981761F0A28DAE0FBF2FB11D5D96F8
:100E50008C91928D9F5F9F73928F90E008958FEF9A
:100E60009FEF0895FC01918D828D981731F0828D4E
:100E7000E80FF11D858D90E008958FEF9FEF0895A5
:100E8000FC01918D228D892F90E0805C9F4F821B09
:100E900091098F739927089585E594E00E94400792
:100EA00021E0892B09F420E0822F089580E090E072
:100EB000892B29F00E944C0781110C9400000895A1
:100EC000FC01A48DA80FB92FB11DA35ABF4F2C91BF
:100ED000848D90E001968F739927848FA689B789B6
:100EE0002C93A089B1898C91837080648C93938DAD
:100EF000848D981306C00288F389E02D80818F7D50
:100F000080830895EF92FF920F931F93CF93DF9307
:100F1000EC0181E0888F9B8D8C8D98131AC0E88935
:100F2000F989808185FF15C09FB7F894EE89FF8904
:100F30006083E889F98980818370806480839FBFA2
:100F400081E090E0DF91CF911F910F91FF90EF90A2
:100F50000895F62E0B8D10E00F5F1F4F0F731127B2
:100F6000E02E8C8D8E110CC00FB607FCFACFE889ED
:100F7000F989808185FFF5CFCE010E946007F1CF0E
:100F8000EB8DEC0FFD2FF11DE35AFF4FF0829FB761
:100F9000F8940B8FEA89FB8980818062CFCFCF9351
:100FA000DF93EC01888D8823B9F0AA89BB89E88991
:100FB000F9898C9185FD03C0808186FD0DC00FB637
:100FC00007FCF7CF8C9185FFF2CF808185FFEDCFB5
:100FD000CE010E946007E9CFDF91CF910895833061
:100FE00081F028F4813099F08230A9F0089587309B
:100FF000A9F08830C9F08430B1F4809180008F7DF1
:1010000003C0809180008F7780938000089584B51D
:101010008F7784BD089584B58F7DFBCF8091B0001C
:101020008F778093B00008958091B0008F7DF9CFC5
:10103000CF93DF93282F30E0F901E654FA4F8491E3
:10104000F901EC50FA4FD491F901EE5EF94FC491D9
:10105000CC23A1F081110E94EF07EC2FF0E0EE0FFE
:10106000FF1FE055FA4FA591B491EC91ED2381E07B
:1010700090E009F480E0DF91CF91089580E090E066
:10108000FACF1F93CF93DF93282F30E0F901E65476
:10109000FA4F8491F901EC50FA4FD491F901EE5EC8
:1010A000F94FC491CC23A9F0162F81110E94EF07AC
:1010B000EC2FF0E0EE0FFF1FE85FF94FA591B49120
:1010C0008FB7F894EC91111108C0D095DE23DC9312
:1010D0008FBFDF91CF911F910895DE2BF8CF109233
:1010E00009041092080410923204109254041092D1
:1010F000300481E080932F0410920A0461E082E1C1
:101100000E94410861E083E10E944108E9EBF0E0C0
:1011100080818E7F808380818D7F808388E480932F
:10112000B80085E48093BC008FED96E090930704AF
:101130008093060480EE96E0909305048093040467
:101140000895CF93DF9390E0FC01EC50FA4F249187
:101150008E5E994FFC0184918823C9F090E0880F3E
:10116000991FFC01E253FA4FA591B491FC01E85F8D
:10117000F94FC591D49161110DC09FB7F8948C912E
:10118000209582238C938881282328839FBFDF9119
:10119000CF910895623051F49FB7F8943C91822F1B
:1011A000809583238C93E8812E2BEFCF8FB7F89413
:1011B000EC912E2B2C938FBFEACF3FB7F894809100
:1011C000D8039091D903A091DA03B091DB0326B53F
:1011D000A89B05C02F3F19F00196A11DB11D3FBF6F
:1011E000BA2FA92F982F8827BC01CD01620F711D3E
:1011F000811D911D42E0660F771F881F991F4A9538
:10120000D1F708958F929F92AF92BF92CF92DF92C3
:10121000EF92FF924B015C010E94DD086B017C01A3
:101220000E94DD086C197D098E099F09683E734094
:1012300081059105A8F321E0821A9108A108B1085F
:1012400088EEC80E83E0D81EE11CF11C81149104C5
:10125000A104B10429F7FF90EF90DF90CF90BF90E9
:10126000AF909F908F9008954115510529F4EAE7BA
:10127000F0E080818F7780836A307105B9F0CB010F
:10128000880F991F880F991F807267706860682B9C
:1012900088E10FB6F894A895809360000FBE609324
:1012A0006000E0E6F0E0808180648083232BD9F445
:1012B00083B7817F846083BFF89483B7816083BFE5
:1012C00085B7806685BF8F7D85BF7894889583B705
:1012D0008E7F83BF7894452B29F4EAE7F0E0808184
:1012E00080688083089583B7817F846083BFF8948A
:1012F00083B7816083BF7894889583B78E7F83BFDF
:101300007894E9CFEF92FF920F931F93CF93DF93DF
:10131000EC01EC80FD806E157F050CF070C057FF6E
:1013200004C0240F351F50E040E08E819F81FA01F8
:10133000E20FF31F8E179F071CF49C01241B350B33
:10134000121613060CF05BC0922F842F869586959B
:1013500086958E9DD0018F9DB00D11246A0F7B1F45
:10136000AF8DB8A1A60FB71F477049F188E0841B65
:10137000482F682F70E0FB01E855FA4FE4912817D9
:1013800008F063C0621B71092FEF30E002C0359591
:1013900027956A95E2F7E2230130110539F0B0F1A3
:1013A0000230110561F58C91E82702C08C91E82B81
:1013B000EC93941720F12C813D81A20FB31FE92FEC
:1013C000E41BE83078F00230110521F58E2F9C9156
:1013D00090959C932C813D81A20FB31F885088303B
:1013E000B0F7E770EE2359F0F0E0E056FA4FE491E1
:1013F00001301105F9F010F10230110519F1DF91FA
:10140000CF911F910F91FF90EF900895E0958C91EF
:10141000E823CECF81E00115110509F480E0819524
:101420009E2F8C932C813D81A20FB31F9850983032
:10143000C0F7D7CF8C91E82BEC93E1CFE0958C915E
:10144000E823FACF8C91E827F7CF0130110509F492
:10145000ADCFE0F20230110509F4A5CFAE0DBF1DEE
:10146000AECF0F931F93CF93DF9377FF04C0260F68
:10147000371F70E060E0DC011496CD91DC91FB0138
:10148000E20FF31FCE17DF071CF49E01261B370B5C
:10149000121613064CF5FA0157FD3796A3E0F595A1
:1014A000E795AA95E1F7EC9FD001ED9FB00DFC9F69
:1014B000B00D11246A0F7B1FDC015F96ED91FC914A
:1014C000E60FF71F4770552781E090E001C0880FB5
:1014D0004A95EAF7482F0130110559F0A8F02E0F70
:1014E0003F1F02301105E1F0DF91CF911F910F9165
:1014F00008952E0F3F1FE217F307B1F38191DF012B
:101500001197842B8C93F7CF80952E0F3F1FE217F6
:10151000F30751F39191DF01119798239C93F7CF33
:10152000E217F30709F38191DF01119784278C9368
:10153000F7CF0F931F93FA01DC0156964C91569703
:101540004230E9F04330A1F1413061F514964D91FC
:101550005C91DA01AE1BBF0BFD01E21BF30B77FDC3
:101560000BC0DC0116964D915C916417750724F44D
:10157000AB01BF010E94310A1F910F91089514968B
:101580004D915C91DA01A61BB70BBD016150710949
:10159000DC0116964D915C91DA01AE1BBF0BFD018B
:1015A000E21BF30B77FDE8CFAF010E948209E4CF85
:1015B00016964D915C91DA01A61BB70BBD016150E7
:1015C0007109CDCF0F931F93FA01DC0156964C9110
:1015D00056974230A9F0433091F1413019F51496F5
:1015E0004D915C91DA01AE1BBF0BFD013197F7FD08
:1015F00004C0AB01BF010E9482091F910F910895A1
:1016000014964D915C91DA01A61BB70BBD01DC016C
:1016100016964D915C91DA01AE1BBF0BFD0131971F
:10162000621B730BF7FDE9CFDC0116964D915C91BF
:10163000E417F50714F7AF010E94310ADECF1696C2
:101640004D915C91DA01A61BB70BBD01621B730BB8
:10165000CECFFC0177FD64C080859185681779073E
:101660000CF05EC057FD5CC0828593854817590712
:101670000CF056C086898230B1F0833029F1813078
:1016800041F484819581841B950BAB01BC016150B1
:1016900071092130310509F108F443C022303105C8
:1016A00009F463C0089584819581DC01A61BB70B02
:1016B000BD016150710986819781DC01A41BB50BC6
:1016C000AD0141505109E5CF86819781861B970B6B
:1016D000BA01AC0141505109DCCFCA0157FD079650
:1016E000A3E095958795AA95E1F7A481B5818A9F96
:1016F00090018B9F300D9A9F300D1124620F731F44
:10170000078CF0A1E02DE60FF71F4770552721E069
:1017100030E001C0220F4A95EAF78081822B808356
:101720000895CA0157FD079633E0959587953A9538
:10173000E1F7A481B5818A9F90018B9F300D9A9F1C
:10174000300D1124620F731F078CF0A1E02DE60FFE
:10175000F71F4770552781E090E001C0880F4A9538
:10176000EAF7809590818923DACFCA0157FD079661
:1017700023E0959587952A95E1F7A481B5818A9F05
:1017800090018B9F300D9A9F300D1124620F731FB3
:10179000078CF0A1E02DE60FF71F4770552721E0D9
:1017A00030E001C0220F4A95EAF780818227B7CF47
:1017B00008958EBD00000DB407FEFDCF8EB50895CF
:1017C0008CBD9DBD08950895FC016370668B848176
:1017D000958126813781613039F0633029F0918716
:1017E0008087338722870895318720879387828770
:1017F00008952F923F924F925F926F927F928F92B5
:101800009F92AF92BF92CF92DF92EF92FF920F938F
:101810001F93CF93DF93CDB7DEB76A970FB6F894D7
:10182000DEBF0FBECDBF9A8F898F7A8369834A014D
:10183000D22E18870F833701BC2CDC0159962D91CD
:101840003C915A972115310509F015C118968D91D3
:101850009C911997681779070CF0D7C11A968D914A
:101860009C91481759070CF0D0C14C2C512CB6E074
:10187000CB9E600D711D11247C876B871616170691
:101880000CF0C3C1EA2DF0E0FA87E98793E0EE0F90
:10189000FF1F9A95E1F7F88BEF87CF01840F951F13
:1018A000181619060CF0B1C1A98DBA8D58968C91F5
:1018B000811104C0BFEABD1508F4D394A98DBA8D77
:1018C000ED91FC9111970284F385E02DCD010995EE
:1018D000B5E0DB9EC0011124E981FA81FC83EB8332
:1018E000312C212C9C0120563F4F388F2F8B4A2DB5
:1018F00050E05E8B4D8BEF89F88DE20DF31D449126
:101900009E828D82D12CC12C69817A81620D731DDA
:101910007A8B698B842F90E09C8B8B8BE98DFA8D71
:10192000A081B18140FF82C0F1E0BF126FC0AF1251
:101930006DC01C96ED91FC912F813885A4014C0D52
:101940005D1D69897A89898D9A8D0995EB89FC8954
:10195000F595E7954E2F5FEFC51AD50A6D817E810B
:101960008D899E89680F791F7E836D8398E0C916E3
:10197000D10481F6AFEF2A1A3A0AEB81FC81E40D1B
:10198000F51DFC83EB83F5E02F16310409F0B3CF8E
:101990002F81388526153705B9F0A98DBA8DED91BF
:1019A000FC91B1E0BB1257C0AB1255C069817A817E
:1019B0006B5F7F4F0088F189E02D830128E030E0E4
:1019C000A401898D9A8D0995A98DBA8DED91FC910F
:1019D00011970688F789E02DCD016A960FB6F89425
:1019E000DEBF0FBECDBFDF91CF911F910F91FF9052
:1019F000EF90DF90CF90BF90AF909F908F907F90AF
:101A00006F905F904F903F902F9009941E96ED91AC
:101A1000FC91EF80F88409851A8592014D815E81E1
:101A20006B817C81898D9A8D099590CF2F81388526
:101A30002615370509F48ACF31E0B31207C0A31287
:101A400005C01C96ED91FC91930178CF1E96ED9107
:101A5000FC917301E0CF6B857C8564197509068460
:101A6000F785E02D73010F8518899201A401898DF6
:101A70009A8D0995A9CFF9013496949132974591A1
:101A80005491D91AB7E0DB9E400D511D1124F90184
:101A9000259134913C8B2B8BFA0125903490FA01DF
:101AA0003296749031963491398B32966490319697
:101AB000449041E04C1518F04A1508F07FC0662D9F
:101AC000062C000C770B7C836B83842D042C000C7C
:101AD000990B9E838D83A98DBA8DED91FC91119701
:101AE0000284F385E02DCD010995512CD12CC12C18
:101AF000EA2DF0E0FA87E9872B2D30E03C872B8731
:101B0000A401440D511D47FC5A95588F4F8B698194
:101B10007A81660D711D67FC7A957E876D8779895C
:101B2000C71608F051CF2C2D30E04D815E81420F59
:101B3000531FA985BA854A9FC0014B9F900D5A9F9C
:101B4000900D1124FC01E80DF91DF88BEF87852D10
:101B5000612C4F89588D420F531F5E8B4D8B67143C
:101B600008F050C044244394480E877041F4C101EA
:101B70000196EB89FC89E20DF31DD4901C01D7FE80
:101B800019C0A98DBA8DED91FC91662D70E0B1E080
:101B9000BB1219C0AB1217C02D853E85620F731F93
:101BA0000484F585E02D2F8138854D895E89898DE6
:101BB0009A8D0995DD0C6394842DD1CF1E821D82F0
:101BC0001C821B8288CF4B815C81640F751FAB85A3
:101BD000BC856A9FC0016B9F900D7A9F900D112468
:101BE00069817A81680F791F0684F785E02DEF807F
:101BF000F88409851A859D014F855889898D9A8DAC
:101C00000995D8CF570CC3948ACF6A960FB6F8942B
:101C1000DEBF0FBECDBFDF91CF911F910F91FF901F
:101C2000EF90DF90CF90BF90AF909F908F907F907C
:101C30006F905F904F903F902F9008958F929F925A
:101C4000AF92CF92EF92FF920F931F93CF93DF93B8
:101C5000EC01262F898D9A8D009709F051C06A30CA
:101C6000D1F41D861C868D8948E0849F9001112443
:101C70008E859F85820F931F9F878E8781E090E0DE
:101C8000DF91CF911F910F91FF90EF90CF90AF9088
:101C90009F908F9008956D3089F3CC88AD888F899F
:101CA0008823C1F08C859D8536E0C39E800D911DF3
:101CB0001124488559854817590764F44E855F8576
:101CC0001D861C8638E0A39EC0011124840F951F39
:101CD0009F878E87EA88FB88088919894E855F85EA
:101CE0006C857D85CE010E94F90B2C898C859D85A4
:101CF00046E0249F800D911D11249D878C87BECFC7
:101D00006A3069F41D861C86FC013696E4912D89A3
:101D10008E859F85E29F800D911D1124ADCF6D3082
:101D200009F4ACCFFC0134963491631708F4A6CFC4
:101D30003196E491E61708F4A1CFFC013296859024
:101D40009490462F431B342F47E0349F800C911C06
:101D50001124F401329634913196E4913323A9F1A0
:101D6000EE2399F1CC88F4013596E491AD884F8942
:101D7000442301F10E2E000CFF0BE30FF11DCE9E4C
:101D8000A001CF9E500D11246C857D85460F571FF5
:101D900068857985641775076CF44E855F851D86A7
:101DA0001C86FC013696E491AE9E400D511D112417
:101DB0005F874E87EA88FB88088919894E855F8589
:101DC0006C857D85CE010E94F90BF4013496E49177
:101DD0002C898C859D85E29F800D911D11248DCFCE
:101DE0006F927F928F929F92AF92BF92CF92DF922B
:101DF000EF92FF920F931F93CF93DF93EC016B0150
:101E00005A0139014801E881F9810284F385E02D06
:101E10000995E881F9810288F389E02D8701930112
:101E2000A501B601CE010995A501480D591D4150E6
:101E30005109E881F9810288F389E02D9301B60107
:101E4000CE010995E881F9810088F189E02D94019E
:101E5000A501B601CE010995C60CD71CB60161508B
:101E60007109E881F9810088F189E02D9401A501CB
:101E7000CE010995E881F9810688F789E02DCE0128
:101E8000DF91CF911F910F91FF90EF90DF90CF9056
:101E9000BF90AF909F908F907F906F9009946F92BA
:101EA0007F928F929F92AF92BF92CF92DF92EF92EA
:101EB000FF920F931F93CF93DF935C01EB016A01B5
:101EC000490138018701DC01ED91FC91621773072C
:101ED00019F5641675062CF0962D872D3A01C92E3A
:101EE000D82E9601261937092F5F3F4F048CF58DA8
:101EF000E02DA301BE01C5010995DF91CF911F918E
:101F00000F91FF90EF90DF90CF90BF90AF909F9098
:101F10008F907F906F9008954615570591F426177E
:101F2000370724F0892D4B01C22FD82F9E01281985
:101F300039092F5F3F4F068CF78DE02DA601B401C4
:101F4000DACF0284F385E02D0995D501ED91FC915E
:101F50000488F589E02D83019401A601BE01C50125
:101F60000995D501ED91FC910688F789E02DC50111
:101F7000DF91CF911F910F91FF90EF90DF90CF9065
:101F8000BF90AF909F908F907F906F900994EF9249
:101F9000FF920F931F93DC011A960D911C911B97D2
:101FA00018962D913C911997ED91FC9100A0F1A10B
:101FB000E02D7B0150E040E070E060E009951F916A
:101FC0000F91FF90EF9008954F925F926F927F92E2
:101FD0008F929F92AF92BF92CF92DF92EF92FF9239
:101FE0000F931F93CF93DF936C012B015A0139019B
:101FF0004801DC01ED91FC910284F385E02D099507
:10200000E201640C751CD601ED91FC91C615D70553
:102010005CF40088F189E02D87019401A501BE01DF
:10202000C60109952196EFCF0688F789E02DC601F4
:10203000DF91CF911F910F91FF90EF90DF90CF90A4
:10204000BF90AF909F908F907F906F905F904F90D8
:1020500009948F929F92AF92BF92CF92DF92EF92AC
:10206000FF920F931F93CF93DF93EC015B014A0123
:102070006901E881F9810284F385E02D09959501D4
:102080002C0D3D1D21503109E881F9810488F58925
:10209000E02D78018401A401B501CE010995E88104
:1020A000F9810688F789E02DCE01DF91CF911F914C
:1020B0000F91FF90EF90DF90CF90BF90AF909F90E7
:1020C0008F9009948F929F92AF92BF92CF92DF929E
:1020D000EF92FF920F931F93CF93DF93EC015B017D
:1020E0004A0169017801E881F9810284F385E02DD4
:1020F0000995C80CD91C860101501109E881F981A4
:102100000488F589E02D9501A401B501CE0109955A
:10211000E881F9810688F789E02DCE01DF91CF9122
:102120001F910F91FF90EF90DF90CF90BF90AF90F5
:102130009F908F900994EF92FF920F931F93DC0171
:10214000ED91FC9100A0F1A1E02D09951F910F9157
:10215000FF90EF9008950F931F93DC01ED91FC9198
:10216000068CF78DE02D09951F910F9108950F931F
:102170001F93DC01ED91FC91048CF58DE02D099508
:102180001F910F910895DC01ED91FC910084F18580
:10219000E02D09943F924F925F926F927F928F92BF
:1021A0009F92AF92BF92CF92DF92EF92FF920F93E6
:1021B0001F93CF93DF9300D000D0CDB7DEB75C0183
:1021C0003B016A014901280187E0480E511C93E058
:1021D000559447949A95E1F7CA018E0D9F1D9A83F5
:1021E0008983F12CE12C312C1C821B828B819C81F8
:1021F00087709927330C892B61F4EB81FC8183E094
:10220000F595E7958A95E1F7EE0DFF1DE80DF91DAF
:10221000349037FE0AC021E030E0A6016B817C815A
:10222000660D771DC5010E94C3108B819C810196AC
:102230009C838B8308171907C9F69FEFC91AD90A1F
:10224000E40CF51C89819A81C816D90669F60F90AD
:102250000F900F900F90DF91CF911F910F91FF90F2
:10226000EF90DF90CF90BF90AF909F908F907F9036
:102270006F905F904F903F9008952F923F924F92B2
:102280005F926F927F928F929F92AF92BF92CF9206
:10229000DF92EF92FF920F931F93CF93DF9300D0C3
:1022A00000D000D0CDB7DEB73C016A013E832D835C
:1022B000FC82EB825801A41AB50AB7FE03C0B194A0
:1022C000A194B1088D809E80861A970A97FE03C05C
:1022D0009194819491088A149B045CF0902F812F33
:1022E0000D811E819D838E839C2D8D2D6B01692F09
:1022F000782F0C151D055CF09D818E817E836D838A
:10230000692F782F902F812F8601C92ED82E160184
:10231000201A310A2B012D813E81421A530A57FEA1
:1023200003C0519441945108710137FE03C03FEF3F
:10233000E31AF30AF594E7948D819E818617970737
:102340005CF5A1E0B0E0BA83A983C016D1064CF1D8
:10235000D301ED91FC910484F585E02D2B813C8126
:10236000A8016D817E818A149B041CF04D815E81E1
:10237000B801C3010995E418F508F7FE0AC02D81DC
:102380003E8189819A81280F391F3E832D83E20C7B
:10239000F31C0F5F1F4FD9CF2FEF3FEF3A832983F5
:1023A000D4CF26960FB6F894DEBF0FBECDBFDF9117
:1023B000CF911F910F91FF90EF90DF90CF90BF9042
:1023C000AF909F908F907F906F905F904F903F90D5
:1023D0002F900895089585ED8093BC008091BC00F6
:1023E00084FDFCCF1092300408952091B003260F95
:1023F0003327331F21323105ECF420913004FC01E6
:1024000090E080E0243069F082E00895A091B0036C
:102410002191AC0140575C4FA40FB52FB11D2C93F7
:102420000196861798F38091B003680F6093B0030C
:1024300080E0089581E00895E09109048091080406
:10244000E81730F4F0E0EC51FC4F808190E0089503
:102450008FEF9FEF089590910904809108042FEF6A
:102460003FEF981748F4E92FF0E0EC51FC4F208142
:1024700030E09F5F90930904C9010895809108049A
:1024800090910904891B990B0895CF92DF92EF92E6
:10249000FF920F931F93CF93DF937C01CB018A01AF
:1024A00020913104222389F0EB016B01C40ED51E6B
:1024B000CC15DD0569F06991D701ED91FC91019092
:1024C000F081E02DC7010995F3CF642F0E94F5112B
:1024D000C801DF91CF911F910F91FF90EF90DF9096
:1024E000CF900895CF93DF931F92CDB7DEB7698366
:1024F000209131042223F9F020915404203258F025
:1025000021E030E0FC013383228390E080E00F90F3
:10251000DF91CF91089580913204E82FF0E0ED5CD7
:10252000FB4F998190838F5F809332048093540492
:1025300081E090E0ECCF61E0CE0101960E94F511C0
:10254000F7CFCF93C72F91E09093310496E3909308
:1025500053041092320410925404682F82EF94E0D6
:102560000E9472126C2F82EF94E00E94721260E05F
:1025700082EF94E00E94721281E0CF910C94820667
:1025800081E00C948206FF920F931F93CF93DF9309
:10259000F82ED92FC62F80911B0590911C0500970E
:1025A00009F452C020911F0531E03093310420938B
:1025B00053041092320410925404DC01ED91FC910A
:1025C0000190F081E02D60E009950F2D1D2FD1E0E5
:1025D000FF24F394C15080911B0590911C05CF3FBF
:1025E00061F1D032C8F00E94C01280911B05909119
:1025F0001C0520911F05F092310420935304109282
:10260000320410925404DC01ED91FC910190F081B0
:10261000E02D60E00995D1E080911B0590911C05AB
:10262000F8016491DC01ED91FC910190F081E02DC5
:102630000995DF5F0F5F1F4FCDCFDF91CF911F91C6
:102640000F91FF900C94C012E0912B05F0912C0596
:102650009081809131058095892380830F2D1D2FD6
:10266000C15008F438C0F8018491209119053091C7
:102670001A05232B29F00E94D90B0F5F1F4FF0CFB3
:1026800028E030E040E8E0912705F091280590919E
:102690002F05582F5423D9F05081952B9083E0912A
:1026A0002905F0912A05908150913005952B908352
:1026B000E0912905F0912A0550819091300590957F
:1026C00095239083469521503109E9F6D6CF508164
:1026D00090959523E3CFDF91CF911F910F91FF90BC
:1026E00008951F93CF93DF93EC018D8D9E8D0097FE
:1026F00021F1162F29A131E03093310420935304A6
:102700001092320410925404DC01ED91FC9101907E
:10271000F081E02D60E009958D8D9E8DDC01ED91BD
:10272000FC910190F081E02D612F09958D8D9E8D9A
:10273000DF91CF911F910C94C012ADA5BEA59C91C5
:102740008BA9809589238C938B8D9C8D892B31F05F
:10275000862FDF91CF911F910C94D90B28E030E0A8
:1027600080E8A9A5BAA599A9462F4823C1F04C91A4
:10277000942B9C93ABA5BCA59C914AA9942B9C93AC
:10278000ABA5BCA54C919AA9909594239C93869552
:102790002150310931F7DF91CF911F9108954C916C
:1027A00090959423E6CFEF92FF920F931F93CF93D0
:1027B000DF9380911B0590911C05892B09F493C030
:1027C00020913505309136054091370550913805F7
:1027D00060E074E284EF90E00E94152220513109FC
:1027E0004109510956954795379527952093B8008B
:1027F00065E086EA9CE00E94C31260910205615088
:102800008EEF94E00E94711320910405309105052C
:10281000C901079697FD079623E0959587952A9518
:10282000E1F72091020530910305829F8001839F8B
:10283000100D929F100D1124C0911D05D0911E0501
:1028400080911B0590911C050C0F1D1F009709F42A
:1028500089C020911F0531E0309331042093530447
:102860001092320410925404DC01ED91FC9101901D
:10287000F081E02D60E40995FF24F394EE24E394C5
:1028800080911B0590911C050C171D0709F442C08F
:10289000BFE1BF15D0F40E94C01280911B0590913A
:1028A0001C0520911F05E0923104209353041092DF
:1028B000320410925404DC01ED91FC910190F081FE
:1028C000E02D60E40995FF24F39480911B0590911D
:1028D0001C056991DC01ED91FC910190F081E02DE6
:1028E0000995F394CDCF8091190590911A05892B04
:1028F00031F080913305909134050E94E00BE09116
:102900002D05F0912E0590818091320580958923C7
:1029100080836ECF0E94C01280911B0590911C0590
:10292000892B09F460C02091390530913A05409116
:102930003B0550913C0560E074E284EF90E00E941A
:10294000152220513109410951095695479537956E
:1029500027952093B800DF91CF911F910F91FF90A1
:10296000EF900895E0912B05F0912C0580819091D6
:102970003105892B80830C171D0771F289912091F5
:10298000190530911A05232B19F00E94D90BF3CFAA
:1029900028E030E040E8E0912705F091280590918B
:1029A0002F05582F5423D9F05081952B9083E09117
:1029B0002905F0912A05908150913005952B90833F
:1029C000E0912905F0912A0550819091300590956C
:1029D00095239083469521503109E9F6CCCF50815B
:1029E00090959523E3CFE0912D05F0912E05808100
:1029F00090913205892B8083AECF1F93CF93DF93C5
:102A0000EC01162F8D8D9E8D892BB1F12FA938AD3C
:102A100049AD5AAD60E074E284EF90E00E94152267
:102A20002051310941095109569547953795279508
:102A30002093B80066EA111167EACE010E94711373
:102A40008D8D9E8D892B41F12BAD3CAD4DAD5EAD95
:102A500060E074E284EF90E00E9415222051310979
:102A60004109510956954795379527952093B80008
:102A7000DF91CF911F9108958B8D9C8D892B21F033
:102A80008DA99EA90E94E00BEFA5F8A990818CA9C1
:102A9000809589238083CECFEFA5F8A980819CA95A
:102AA000892B8083E5CF90E080E00895CF93DF937A
:102AB000C5E0D0E061E085E00E94410861E086E089
:102AC0000E94410860E971E080E090E00E94020904
:102AD00060E085E00E94410860E086E00E944108D5
:102AE00060E971E080E090E00E940209219711F70F
:102AF000DF91CF910895CF92DF92EF92FF920F93E3
:102B00001F93CF93DF938C0187E0E82E81E0F82EAE
:102B1000C80186549A4F6C01F701C191D1917F0190
:102B200061E0802F0E94A108209729F460E0802FA7
:102B30000E94410826C0CF3FD10511F461E0F7CFD4
:102B4000F60184918330B9F140F48130B1F08230E4
:102B500069F1C038D10594F7E9CF8730B1F18830F9
:102B6000E1F18430B1F78091800080628093800031
:102B7000D0938B00C0938A0004C084B5806884BD64
:102B8000C7BD6CE070E080E090E00E940209FBE2CB
:102B9000EF16F3E0FF0609F0BFCFDF91CF911F9151
:102BA0000F91FF90EF90DF90CF90089584B58062F1
:102BB00084BDC8BDE6CF809180008068809380008E
:102BC000D0938900C0938800DCCF8091B0008068EA
:102BD0008093B000C093B300D4CF8091B0008062E6
:102BE0008093B000C093B400CCCF85E090E00E9409
:102BF0007B1560E082E00E9441081092DE03089598
:102C0000CF9391E09093310496E390935304109204
:102C1000320410925404682F82EF94E00E947212E2
:102C200080E00E948206809130048111FCCF81E017
:102C30008093300480932F049FEF90932E04109282
:102C40002D0480932C0480930B0480910B048C66DC
:102C500080930B0480910A04813099F510920A0444
:102C600080910B048093BB008091BC0083FDF8CF62
:102C700085EC8093BC00809130048130E1F3809139
:102C80002D0492E0823010F490912D04ACE0B4E079
:102C9000E4EEF3E080E0891316C0109209048093FB
:102CA000080482EF94E00E942B12C82F82EF94E078
:102CB0000E942B1220E03C2F820F932F911DCF9169
:102CC000089585EED6CF2D9121938F5FE4CFCF92DB
:102CD000DF92EF92FF920F931F93CF93DF9384E0E5
:102CE0000E940016EC01BC017727072E000C880B10
:102CF000990B0E94EE2020E030E040E85BE30E9468
:102D0000A3216B017C016D2F70E090E080E00E94B8
:102D1000EC209B01AC01C701B6010E94D31F0E94A9
:102D2000B6208091E103882351F03EE0E32EF12CA0
:102D300000E110E024E830E06436710531F590914F
:102D4000E0039923B1F02EE0E22EF12C00E110E037
:102D500024E830E06436710549F481110FC08EE03B
:102D6000E82EF12C00E110E028E630E040E150E0F0
:102D70000EC08823A9F06436710591F49EE0E92E17
:102D8000F12C00E110E028E630E050E040E066E79A
:102D900070E08EEF94E00E94CA1081E08093DF0320
:102DA000DF91CF911F910F91FF90EF90DF90CF9027
:102DB00008952091040530910505C901079697FDF6
:102DC000079623E0959587952A95E1F720910205CE
:102DD00030910305829FA001839F500D929F500D5B
:102DE000112470E060E080911D0590911E050C9407
:102DF00067230E94D9160E94D3131092DF0308950F
:102E00000E946223FB0101900020E9F73197AF0196
:102E1000461B570BDC01ED91FC910280F381E02D04
:102E200009948F929F92AF92BF92EF92FF920F936D
:102E30001F93CF93DF93CDB7DEB7A1970FB6F8946A
:102E4000DEBF0FBECDBF7C01FA01CB0119A222303B
:102E500008F42AE08E010F5D1F4F822E912CB12CB9
:102E6000A12CBF01A50194010E941522F901CA01FC
:102E70006A300CF5605DD8016E938D01232B242BF5
:102E8000252B79F790E080E0109721F0BD01C70174
:102E90000E940217A1960FB6F894DEBF0FBECDBFF9
:102EA000DF91CF911F910F91FF90EF90BF90AF9066
:102EB0009F908F900895695CDECF2F923F924F9242
:102EC0005F926F927F928F929F92AF92BF92CF92BA
:102ED000DF92EF92FF921F93CF93DF93EC016A0191
:102EE0007B01722EAB019601CB01B6010E9410222C
:102EF0006BE773E0811126C046015701E894B7F8EB
:102F00002FEF3FEF4FE75FE7C501B4010E941022AA
:102F100081110CC02FEF3FEF4FE75FE7C501B40110
:102F20000E943F206FE773E0181664F02FEF3FEF29
:102F30004FE75FE4C701B6010E949E211816B4F462
:102F400063E873E0CE01DF91CF911F91FF90EF9086
:102F5000DF90CF90BF90AF909F908F907F906F90B9
:102F60005F904F903F902F900C9402172FEF3FEF00
:102F70004FE75FECC701B6010E943F2087FDE0CF1D
:102F800020E030E0A901C701B6010E943F20312CAA
:102F9000212C87FF0DC0E881F9810190F081E02D9F
:102FA0006DE2CE0109951C01F7FAF094F7F8F09460
:102FB00010E060E070E080E09FE3711641F020E0F7
:102FC00030E040E251E40E9444201F5FF6CFA701A9
:102FD00096010E94D31F2B013C010E94BD204B0192
:102FE0005C012AE0BC01A401CE010E9411177C0102
:102FF000E20CF31C1123E1F1C501B4010E94EC20A5
:103000009B01AC01C301B2010E94D21F4B015C01C4
:10301000E881F9810190F081E02D6EE2CE01099501
:10302000E80EF91E115020F120E030E040E251E4BA
:10303000C501B4010E94A3212B013C010E94BD20C7
:103040004B01B12CA12C2AE0B501A401CE010E94B4
:103050001117E80EF91EC501B4010E94EC209B0176
:10306000AC01C301B2010E94D21F4B015C01DACF57
:10307000C701DF91CF911F91FF90EF90DF90CF902C
:10308000BF90AF909F908F907F906F905F904F9088
:103090003F902F9008951F920F920FB60F92112418
:1030A0002F933F934F935F936F937F938F939F9350
:1030B000AF93BF93EF93FF9385E594E00E94600781
:1030C000FF91EF91BF91AF919F918F917F916F9100
:1030D0005F914F913F912F910F900FBE0F901F90D6
:1030E00018951F920F920FB60F9211242F938F9362
:1030F0009F93EF93FF93E0916504F09166048081C4
:10310000E0916B04F0916C0482FD1BC09081809172
:103110006E048F5F8F7320916F04821741F0E091EE
:103120006E04F0E0EB5AFB4F958F80936E04FF9195
:10313000EF919F918F912F910F900FBE0F901F9045
:1031400018958081F4CF1F920F920FB60F92112421
:103150002F933F938F939F93AF93BF938091D4030B
:103160009091D503A091D603B091D7033091D303AA
:1031700023E0230F2D3758F50196A11DB11D209393
:10318000D3038093D4039093D503A093D603B09335
:10319000D7038091D8039091D903A091DA03B0911D
:1031A000DB030196A11DB11D8093D8039093D90331
:1031B000A093DA03B093DB03BF91AF919F918F91FE
:1031C0003F912F910F900FBE0F901F90189526E8FA
:1031D000230F0296A11DB11DD2CF1F920F920FB6E1
:1031E0000F9211248F930FB6F894A89580916000E8
:1031F000886180936000109260000FBE8F910F90E5
:103200000FBE0F901F9018951F920F920FB60F923E
:1032100011242F933F934F935F936F937F938F93DB
:103220009F93AF93BF93EF93FF938091B900887FF3
:10323000803609F44AC0F0F5883209F4A7C018F5C1
:10324000803109F49BC0B8F4882309F4F9C08830B0
:1032500009F494C0FF91EF91BF91AF919F918F912D
:103260007F916F915F914F913F912F910F900FBE82
:103270000F901F901895883109F488C0803251F75B
:1032800080932E0414C0803409F49DC040F4803330
:10329000B9F38833F9F680932E0485ECB0C08035FD
:1032A00009F485C0883509F496C0883499F60E94DF
:1032B000EB11D0CF883909F48CC038F5883729F064
:1032C00050F4883611F0803729F683E0809330047B
:1032D0001092D20357C0883809F47BC0803919F0A6
:1032E000803809F0B7CF8091D203803208F071C0E6
:1032F000E091D20381E08E0F8093D2038091BB00D6
:10330000F0E0EE54FC4F80833DC0803B39F0E0F4A8
:10331000803A09F479C0883A09F09CCF84E0809320
:1033200030041092B1031092B003E0910604F091C2
:10333000070409958091B00381110FC081E080934B
:10334000B0031092900309C0803C09F4A6CF883CDA
:1033500009F4A3CF883B09F07DCFE091B10381E070
:103360008E0F8093B103F0E0E057FC4F8081809393
:10337000BB009091B1038091B00329C080910B04F0
:103380008093BB0085EC8093BC0064CF90912D04AA
:1033900080912C04981758F5E0912D0481E08E0F50
:1033A00080932D04F0E0E45FFB4F8081E9CFE09152
:1033B0002D0481E08E0F80932D048091BB00F0E0FE
:1033C000E45FFB4F808390912D0480912C0498172B
:1033D000C8F285E8D8CFE0912D0481E08E0F80936C
:1033E0002D048091BB00F0E0E45FFB4F808380916F
:1033F0002F0481115CCF81E080930A0484EA8093DA
:10340000BC001092300426CF85EC8093BC00109253
:1034100030048091D203803230F4E091D203F0E0A6
:10342000EE54FC4F10826091D20370E0E0910404EE
:10343000F091050482EB93E009951092D2030ACF34
:1034400010922E0434CFE5E5F4E01382128248EEA8
:1034500053E060E070E044835583668377838FE2B6
:1034600093E09183808385EC90E09587848784EC5A
:1034700090E09787868780EC90E0918B808B81EC41
:1034800090E0938B828B82EC90E0958B848B86EC22
:1034900090E0978B868B118E128E138E148EA2EF76
:1034A000B4E013961C921E92129714964D935D935E
:1034B0006D937C93179781E493E011969C938E9380
:1034C00040E050E060EA7FE340933D0550933E05C5
:1034D00060933F0570934005EEEFF4E01382128293
:1034E00020E830E03583248380E290E09783868370
:1034F0003187208793878287168A158614861786D8
:10350000168681E0858B848B2FEF3FEF338B228BE8
:10351000318B208B878B108E128E118E83E593E07A
:1035200091838083148E138EB68FA58F10A2178E71
:103530008FEF84A385A386A387A380A780E585ABAF
:1035400016AA80E89AE1A6E0B0E087AB90AFA1AF01
:10355000B2AF80EA96E8A1E0B0E083AF94AFA5AF48
:10356000B6AF0895789484B5826084BD84B58160D7
:1035700084BD85B5826085BD85B5816085BD80913E
:103580006E00816080936E001092810080918100B6
:1035900082608093810080918100816080938100AE
:1035A000809180008160809380008091B100846070
:1035B0008093B1008091B00081608093B0008091D1
:1035C0007A00846080937A0080917A008260809390
:1035D0007A0080917A00816080937A0080917A00ED
:1035E000806880937A001092C10064E670E080E009
:1035F00090E00E94020988E199E20FB6F894A8953C
:10360000809360000FBE9093600080911D059091A3
:103610001E05892B39F10E94D916809104059091DD
:1036200005056091020570910305813291050CF04A
:103630005EC2AC014052510957FF02C04F5F5F4F5D
:10364000559547956357710977FF02C06F5F7F4FAC
:103650007595679590E2E92EF12C03E710E026E2DC
:1036600036E05DC22091040530910505C901079639
:1036700097FD0796A3E095958795AA95E1F7209188
:10368000020530910305AC01429FC001439F900D9C
:10369000529F900D11240E943D2290931E0580930D
:1036A0001D05892B09F0B7CF0E94D91681E090E063
:1036B000909311058093100590930F0580930E054C
:1036C0000E946F08E0916504F091660482E08083B7
:1036D000E0916104F09162041082E0916304F09142
:1036E00064048FEC808310926D04E0916904F09182
:1036F0006A0486E08083E0916704F0916804808129
:1037000080618083E0916704F09168048081886023
:103710008083E0916704F0916804808180688083F1
:10372000E0916704F091680480818F7D808360E080
:103730008EE00E94A10860E08FE00E94A10860E096
:1037400080E10E94A10861E082E00E94A10861E09E
:1037500085E00E94A10861E086E00E94A10862E085
:1037600083E00E94A10862E084E00E94A10860E07A
:1037700082E00E9441080E94F91668EC70E080E047
:1037800090E00E9402090E946F0860E074E58EEFED
:103790000E94A11260E070E486E00E94A112C0E0E5
:1037A000D0E06EE1C62ED12C7AE0A72EB12C64E6D3
:1037B00070E080E090E00E94020964E873E080E03D
:1037C00090E00E94020982E00E94001654E0969563
:1037D00087955A95E1F7BC0190E080E00E94EC20CB
:1037E00020913D0530913E0540913F0550914005A7
:1037F0000E94A32120E030E04AE754E40E944420E4
:10380000AB01BC0122E085E594E00E945D1767E80A
:1038100073E085E594E00E940217A89583E00E947A
:103820001808892BD1F47090DE03711006C08091C6
:10383000E2039091E303892B31F06CEB72E080E0BE
:1038400090E00E94020983E00E941808892B29F465
:10385000772009F42CC30E94F51584E00E94180813
:10386000892B59F58091DE03811106C08091E20316
:103870009091E303892B31F06CEB72E080E090E0F3
:103880000E94020984E00E941808892BB1F48091FB
:103890000001882309F425C386E090E00E947B158F
:1038A0008091E2039091E3038230910508F012C306
:1038B00001969093E3038093E2038FE00E9418083F
:1038C000019709F011C364E670E080E090E00E9487
:1038D00002098FE00E941808019719F481E0809393
:1038E000E10380E10E941808019709F000C364E633
:1038F00070E080E090E00E94020980E10E941808D8
:10390000019719F481E08093E00382E00E940016A1
:1039100044E0969587954A95E1F7BC0190E080E0F8
:103920000E94EC2020913D0530913E0540913F05DD
:10393000509140050E94A32120E030E04AE754E482
:103940000E9444202AE939E949E550E40E949E2179
:1039500018160CF0CFC281E0809300018091E20341
:103960009091E303892B09F482C0809100018823A0
:1039700009F47DC00E94D91630E2E32EF12C08E74D
:1039800010E026EC3AE050E040E070E060E08EEFBE
:1039900094E00E94CA1082E0809312058093130580
:1039A000D0920B05C0920A05B0920D05A0920C05AD
:1039B000109211051092100510920F0510920E052D
:1039C0008091E2039091E3038130910509F0A2C256
:1039D00084E00E9400163C01BC017727072E000CF2
:1039E000880B990B0E94EE2020E030E040E85BE37A
:1039F0000E94A3211B012C01672D70E090E080E064
:103A00000E94EC209B01AC01C201B1010E94D31FB6
:103A10000E94B6202B01770F660877082AE0B301D1
:103A2000A20177FE0DC06DE28EEF94E00E941E0EA3
:103A300044275527BA0144195509660977092AE030
:103A40008EEF94E00E9411176AE873E08EEF94E025
:103A50000E94021767E873E08EEF94E00E9402175D
:103A60000E9467160E94D31381E08093DF03809148
:103A7000E103811105C08091E003882309F474C239
:103A80008091E2039091E303892B09F06DC20E94BB
:103A9000D9160E9467160E94D31381E08093DF033A
:103AA0008091DE03811118C08091E2039091E303BD
:103AB000892B91F48091E10381110EC08091E00384
:103AC00081110AC030E020E050E040E066E070E0A4
:103AD0008DED93E00E943409209709F468CE0E948E
:103AE0004C07882309F463CE0E94000060CEAC012D
:103AF0004054510957FF02C04F5F5F4F559547959E
:103B00006255710977FF02C06F5F7F4F75956795AA
:103B1000E0E4EE2EF12C02E510E026E038E08EEF36
:103B200094E00E94CA1082E08093200580911B05DA
:103B300090911C05892B09F4AFC08CE380931F057D
:103B40000E946F088091260587FD1EC061E00E94DB
:103B5000A10861E0809126050E94410861E070E0C3
:103B600080E090E00E94020960E0809126050E94BA
:103B700041086AE070E080E090E00E94020961E0A4
:103B8000809126050E94410880911B0590911C059B
:103B9000892B09F440C120913505309136054091BB
:103BA00037055091380560E074E284EF90E00E94A0
:103BB00015222051310941095109569547953795EC
:103BC00027952093B80064E080EF95E00E94C3122F
:103BD0006091040561508EEF94E00E94711364E0DF
:103BE0008CEE95E00E94C3128091200564E1813043
:103BF00009F460E18EEF94E00E94711364E088EEB6
:103C000095E00E94C31280910205909103058038CF
:103C1000910509F02BC18091040590910505803232
:103C2000910509F00FC164E084EE95E00E94C31293
:103C300069ED8EEF94E00E9471138091200561EF91
:103C4000813009F462E28EEF94E00E94711366E025
:103C500088ED95E00E94C31280911B0590911C0590
:103C6000892B09F41AC12091390530913A05409108
:103C70003B0550913C0560E074E284EF90E00E94C7
:103C8000152220513109410951095695479537951B
:103C900027952093B80008CD61E0809124050E940B
:103CA000A10861E0809125050E94A108809124056A
:103CB000082E000C990BFC01EE5EF94FE491F0E048
:103CC000EE0FFF1FE85FF94F2591349130932C05DB
:103CD00020932B05FC01EC50FA4FE491E093310561
:103CE00080912505082E000C990BFC01EE5EF94F22
:103CF000E491F0E0EE0FFF1FE85FF94FA591B4915A
:103D0000B0932E05A0932D05FC01EC50FA4FE491E1
:103D1000E09332058C91E82BEC93809119059091FA
:103D20001A05892B09F434C0CFB7F8948091DC03CD
:103D3000811127C0ECE1F6E08491EEEFF5E094917B
:103D4000E82FF0E0EE0FFF1FE253FA4FA591B49178
:103D5000EC91E92321F461E08AE00E94410861E0EE
:103D60008AE00E94A1088CB580618CBD8CB580640E
:103D70008CBD61E08DE00E94A10861E08BE00E94B3
:103D8000A1088091DC038F5F8093DC03CFBFDACE84
:103D900061E0809122050E94A10861E080912305E5
:103DA0000E94A10880912205082E000C990BFC01AD
:103DB000EE5EF94FE491F0E0EE0FFF1FE85FF94F80
:103DC000259134913093280520932705FC01EC5070
:103DD000FA4FE491E0932F0580912305082E000C03
:103DE000990BFC01EE5EF94FE491F0E0EE0FFF1F3E
:103DF000E85FF94FA591B491B0932A05A0932905E6
:103E0000FC01EC50FA4FE491E09330058C91E09581
:103E1000E823EC9397CE8091190590911A05892B90
:103E200031F080913305909134050E94E00BE091D0
:103E30002D05F0912E059081809132058095892382
:103E40008083C1CE8034910509F0F2CE63E081EE2B
:103E500095E00E94C312809120056FEC813009F437
:103E60006FE98EEF94E00E947113E2CE80369105E7
:103E700009F0DECE8091040590910505409709F088
:103E8000D7CE63E08EED95E00E94C31280912005AD
:103E90006FEA813031F760E1E4CFE0912D05F091D8
:103EA0002E05808190913205892B8083FDCB8091F6
:103EB0000001882361F085E090E00E947B1561E0BD
:103EC00082E00E94410881E08093DE03C6CC0E941C
:103ED0005615C3CC0E94F9161092E3031092E20328
:103EE000ECCC0E945615E9CC1092E103FACC10926A
:103EF000E0030BCD109200018091DE03882309F4CA
:103F00002DCD0E94F5151092E3031092E2030E945A
:103F1000F91624CD029709F0A3CD82E00E94001685
:103F200024E0969587952A95E1F7BC0190E080E022
:103F30000E94EC2020913D0530913E0540913F05C7
:103F4000509140050E94A32120E030E04AE754E46C
:103F50000E944420AB01BC0122E08EEF94E00E945D
:103F60005D176CE873E072CD8091DF03882309F45C
:103F700097CD8091E2039091E303892B09F090CDD6
:103F80000E94F9168DCD83E593E09093FF04809312
:103F9000FE0480911D0590911E05009711F00C9470
:103FA000D92208955058BB27AA270E94EA1F0C94D3
:103FB00064210E94562138F00E945D2120F039F4DE
:103FC0009F3F19F426F40C9453210EF4E095E7FB7F
:103FD0000C944D21E92F0E94752158F3BA176207FE
:103FE00073078407950720F079F4A6F50C949721C0
:103FF0000EF4E0950B2EBA2FA02D0B01B901900104
:104000000C01CA01A0011124FF27591B99F0593F47
:1040100050F4503E68F11A16F040A22F232F342F8F
:104020004427585FF3CF469537952795A795F040DD
:104030005395C9F77EF41F16BA0B620B730B840BF2
:10404000BAF09150A1F0FF0FBB1F661F771F881FAA
:10405000C2F70EC0BA0F621F731F841F48F4879502
:1040600077956795B795F7959E3F08F0B0CF9395F4
:10407000880F08F09927EE0F9795879508950E946D
:10408000292108F481E008950E9458200C946421AD
:104090000E945D2158F00E94562140F029F45F3FB4
:1040A00029F00C944D2151110C9498210C9453211A
:1040B0000E94752168F39923B1F3552391F3951B61
:1040C000550BBB27AA2762177307840738F09F5F39
:1040D0005F4F220F331F441FAA1FA9F335D00E2EA6
:1040E0003AF0E0E832D091505040E695001CCAF713
:1040F0002BD0FE2F29D0660F771F881FBB1F2617D6
:1041000037074807AB07B0E809F0BB0B802DBF01AC
:10411000FF2793585F4F3AF09E3F510578F00C947B
:104120004D210C9498215F3FE4F3983ED4F386959B
:1041300077956795B795F7959F5FC9F7880F911D9C
:104140009695879597F90895E1E0660F771F881F88
:10415000BB1F621773078407BA0720F0621B730B3B
:10416000840BBA0BEE1F88F7E09508950E94BD20DE
:104170006894B1110C94982108950E947D2188F0D3
:104180009F5798F0B92F9927B751B0F0E1F0660F1B
:10419000771F881F991F1AF0BA95C9F714C0B1305C
:1041A00091F00E949721B1E008950C949721672F18
:1041B000782F8827B85F39F0B93FCCF3869577958B
:1041C0006795B395D9F73EF4909580957095619574
:1041D0007F4F8F4F9F4F0895E89409C097FB3EF49F
:1041E00090958095709561957F4F8F4F9F4F992344
:1041F000A9F0F92F96E9BB279395F69587957795C2
:104200006795B795F111F8CFFAF4BB0F11F460FF81
:104210001BC06F5F7F4F8F4F9F4F16C0882311F0D9
:1042200096E911C0772321F09EE8872F762F05C0ED
:10423000662371F096E8862F70E060E02AF09A9588
:10424000660F771F881FDAF7880F9695879597F97D
:104250000895990F0008550FAA0BE0E8FEEF161617
:104260001706E807F907C0F012161306E407F5076A
:1042700098F0621B730B840B950B39F40A2661F0DE
:10428000232B242B252B21F408950A2609F4A14081
:10429000A6958FEF811D811D089597F99F6780E88E
:1042A00070E060E008959FEF80EC089500240A9488
:1042B0001616170618060906089500240A94121601
:1042C0001306140605060895092E0394000C11F434
:1042D000882352F0BB0F40F4BF2B11F460FF04C0E1
:1042E0006F5F7F4F8F4F9F4F089557FD9058440F3A
:1042F000551F59F05F3F71F04795880F97FB991F45
:1043000061F09F3F79F08795089512161306140601
:10431000551FF2CF4695F1DF08C01616170618068E
:10432000991FF1CF86957105610508940895E89469
:10433000BB2766277727CB0197F908950E9429218B
:1043400008F48FEF08950E94B6210C9464210E9416
:10435000562138F00E945D2120F0952311F00C9435
:104360004D210C94532111240C9498210E94752105
:1043700070F3959FC1F3950F50E0551F629FF001B8
:10438000729FBB27F00DB11D639FAA27F00DB11DD1
:10439000AA1F649F6627B00DA11D661F829F22275A
:1043A000B00DA11D621F739FB00DA11D621F839FE1
:1043B000A00D611D221F749F3327A00D611D231FB7
:1043C000849F600D211D822F762F6A2F11249F5705
:1043D00050409AF0F1F088234AF0EE0FFF1FBB1F08
:1043E000661F771F881F91505040A9F79E3F5105C7
:1043F00080F00C944D210C9498215F3FE4F3983E9B
:10440000D4F3869577956795B795F795E7959F5F70
:10441000C1F7FE2B880F911D9695879597F9089502
:104420000E942921880B990B0895A1E21A2EAA1B3C
:10443000BB1BFD010DC0AA1FBB1FEE1FFF1FA21754
:10444000B307E407F50720F0A21BB30BE40BF50B51
:10445000661F771F881F991F1A9469F760957095DA
:10446000809590959B01AC01BD01CF010895EE0FA1
:10447000FF1F0590F491E02D09940F931F93CF93A4
:10448000DF938230910510F482E090E0E0914305E3
:10449000F091440530E020E0B0E0A0E0309799F4DE
:1044A0002115310509F44AC0281B390B2430310588
:1044B000D8F58A819B816115710589F1FB01938390
:1044C0008283FE0111C0408151810281138148170E
:1044D0005907E0F04817590799F4109761F01296C0
:1044E0000C93129713961C933296CF01DF91CF91C4
:1044F0001F910F9108950093430510934405F4CF45
:104500002115310551F04217530738F0A901DB019D
:104510009A01BD01DF01F801C1CFEF01F9CF9093FE
:10452000440580934305CDCFFE01E20FF31F819335
:1045300091932250310939832883D7CF20914105A7
:1045400030914205232B41F4209103013091040165
:1045500030934205209341052091010130910201E1
:104560002115310541F42DB73EB740910501509119
:104570000601241B350BE0914105F0914205E2173D
:10458000F307A0F42E1B3F0B2817390778F0AC0176
:104590004E5F5F4F2417350748F04E0F5F1F509353
:1045A000420540934105819391939FCFF0E0E0E075
:1045B0009CCFCF93DF930097E9F0FC0132971382F1
:1045C0001282A0914305B0914405ED0130E020E056
:1045D0001097A1F420813181820F931F2091410512
:1045E000309142052817390709F061C0F093420560
:1045F000E0934105DF91CF910895EA01CE17DF07DF
:10460000E8F54A815B819E0141155105B1F7E90149
:10461000FB83EA8349915991C40FD51FEC17FD071D
:1046200061F4808191810296840F951FE90199833D
:104630008883828193819B838A83F0E0E0E01296F5
:104640008D919C9113970097B9F52D913C911197FD
:10465000CD010296820F931F2091410530914205B2
:104660002817390739F6309751F510924405109202
:104670004305B0934205A0934105BCCFD383C283C9
:1046800040815181840F951FC817D90761F44E5F8F
:104690005F4F88819981480F591F518340838A81D8
:1046A0009B81938382832115310509F0B0CFF0936C
:1046B0004405E09343059ECFFD01DC01C0CF13828A
:1046C0001282D7CF81E090E0F8940C946E23DC0145
:1046D00001C06D9341505040E0F7089516E0C7E5E2
:1046E000D6E004C0FE010E9437222196C835D107CA
:0646F000C9F7F894FFCFAA
:1046F60001000045058000000000000000000000E9
:1047060000000000000000000000000000000001A2
:104716000001000100010001000200020002000287
:104726000003000300040004000400050005000661
:104736000006000700070008000800090009000A33
:10474600000B000B000C000D000E000F00100011F6
:104756000012001300140015001600180019001AA4
:10476600001C001D001E002000210023002500263D
:104776000028002A002C002E0030003100340036BC
:104786000038003A003C003F004100430046004923
:10479600004B004E0050005300560059005C005F6D
:1047A600006200650069006C007000740078007C8F
:1047B600007F00830088008B009000940098009C86
:1047C60000A000A400A800AC00B100B500B900BD6F
:1047D60000C000C400C800CC00D000D300D700DA67
:1047E60000DD00E000E300E600E900EC00EE00F08A
:1047F60000F200F400F600F800F900FA00FB00FCF5
:1048060000FD00FD00FD00FD00FD00FD00FD00FDBA
:1048160000FD00FD00FC00FC00FB00F900F800F7BD
:1048260000F500F300F100EF00EC00EA00E700E419
:1048360000E100DE00DB00D800D400D000CD00C9C6
:1048460000C500C200BE00BA00B600B200AE00A9A4
:1048560000A500A1009D009900950091008D00899A
:1048660000850081007D007900750071006E006A88
:10487600006600620060005D005900570054005158
:10488600004E004C0049004700440041003F003DF7
:10489600003A00380036003400320030002E002C7A
:1048A600002A002800270025002300220020001FE0
:1048B600001D001C001A001900180017001500142E
:1048C6000013001200110010000F000E000D000C66
:1048D600000C000B000A0009000900080008000788
:1048E6000007000600060005000500040004000499
:1048F60000030003000200020002000100010001A3
:10490600000100010001000000000000000000009E
:10491600000000000000000000000000000000820F
:1049260007E2060F07CF0740071E07320700000001
:1049360000721245125315E1063E122B121C12008C
:104946000000001E0EE2065315EA11290BE106C30C
:10495600109B10B710AB103D11E106E40BFD149946
:104966000AE20AE40FC70F4F0FF00E6E616E006980
:104976006E66006F7666000D0A0025002056000060
:107800000C94343C0C94513C0C94513C0C94513CE1
:107810000C94513C0C94513C0C94513C0C94513CB4
:107820000C94513C0C94513C0C94513C0C94513CA4
:107830000C94513C0C94513C0C94513C0C94513C94
:107840000C94513C0C94513C0C94513C0C94513C84
:107850000C94513C0C94513C0C94513C0C94513C74
:107860000C94513C0C94513C11241FBECFEFD8E036
:10787000DEBFCDBF11E0A0E0B1E0ECE9FFE702C060
:1078800005900D92A230B107D9F712E0A2E0B1E065
:1078900001C01D92AD30B107E1F70E942D3D0C945F
:1078A000CC3F0C94003C982F959595959595959582
:1078B000905D8F708A307CF0282F295A8091C0000B
:1078C00085FFFCCF9093C6008091C00085FFFCCF60
:1078D0002093C6000895282F205DF0CF982F809127
:1078E000C00085FFFCCF9093C6000895EF92FF92F1
:1078F0000F931F93EE24FF2487018091C00087FD22
:1079000017C00894E11CF11C011D111D81E4E8164B
:1079100082E4F8068FE0080780E0180770F3E09132
:107920000401F091050109958091C00087FFE9CF1E
:107930008091C6001F910F91FF90EF9008950E94D3
:10794000763C982F8091C00085FFFCCF9093C600B5
:1079500091362CF490330CF09053892F089597555D
:10796000892F08951F930E949F3C182F0E949F3CCF
:107970001295107F810F1F9108951F93182F882350
:1079800021F00E94763C1150E1F71F9108951F935A
:10799000182F0E94763C803249F0809103018F5F5E
:1079A000809303018530C1F01F9108958091C0003C
:1079B00085FFFCCF84E18093C6008091C00085FFE5
:1079C000FCCF1093C6008091C00085FFFCCF80E102
:1079D0008093C6001F910895E0910401F091050184
:1079E00009951F9108950E94763C803241F0809164
:1079F00003018F5F80930301853081F008958091AA
:107A0000C00085FFFCCF84E18093C6008091C00058
:107A100085FFFCCF80E18093C6000895E0910401CA
:107A2000F09105010995089540E951E08823A1F0FE
:107A30002D9A28EE33E0FA013197F1F721503040CA
:107A4000D1F72D9828EE33E0FA013197F1F7215064
:107A50003040D1F7815061F708953F924F925F9285
:107A60006F927F928F929F92AF92BF92CF92DF924E
:107A7000EF92FF920F931F93CF93DF93000080E16B
:107A80008093C4001092C50088E18093C10086E015
:107A90008093C2005098589A259A81E00E94143D24
:107AA00024E1F22E9EE1E92E85E9D82E0FE0C02ECA
:107AB00010E1B12EAA24A394B1E49B2EA6E58A2E50
:107AC000F2E57F2EE0E26E2E79E4572E63E5462E36
:107AD00050E5352E0E94763C8033B1F18133B9F107
:107AE000803409F46FC0813409F476C0823409F41B
:107AF00085C0853409F488C0803531F1823521F1A3
:107B0000813511F1853509F485C0863509F48DC0BC
:107B1000843609F496C0843709F403C1853709F423
:107B200072C1863709F466C0809103018F5F80932C
:107B30000301853079F6E0910401F0910501099582
:107B40000E94763C803351F60E94F33CC3CF0E94E2
:107B5000763C803249F78091C00085FFFCCFF092DF
:107B6000C6008091C00085FFFCCF9092C600809136
:107B7000C00085FFFCCF8092C6008091C00085FFC9
:107B8000FCCF7092C6008091C00085FFFCCF609250
:107B9000C6008091C00085FFFCCF5092C600809146
:107BA000C00085FFFCCF4092C6008091C00085FFD9
:107BB000FCCF3092C6008091C00085FFFCCFB09210
:107BC000C60088CF0E94763C863808F4BDCF0E945C
:107BD000763C0E94F33C7ECF0E94763C803809F4CC
:107BE0009CC0813809F40BC1823809F43CC1883942
:107BF00009F48FC080E00E94C73C6CCF84E10E94F2
:107C0000BD3C0E94F33C66CF85E00E94BD3C0E94D3
:107C1000F33C60CF0E94763C809306010E94763C44
:107C2000809307010E94F33C55CF0E94763C80333D
:107C300009F41DC183E00E94BD3C80E00E94C73C66
:107C400049CF0E94763C809309020E94763C809343
:107C5000080280910C028E7F80930C020E94763C79
:107C6000853409F415C18091080290910902892B8D
:107C700089F000E010E00E94763CF801E85FFE4FDA
:107C800080830F5F1F4F80910802909109020817AF
:107C9000190788F30E94763C803209F045CF809125
:107CA0000C0280FF01C16091060170910701660F0F
:107CB000771F7093070160930601A0910802B091AD
:107CC00009021097C9F0E8E0F1E09B01AD014E0F09
:107CD0005F1FF999FECF32BD21BD819180BDFA9A17
:107CE000F99A2F5F3F4FE417F50799F76A0F7B1F4B
:107CF00070930701609306018091C00085FFFCCF5F
:107D0000F092C6008091C00085FFFCCFB092C60003
:107D1000E1CE83E00E94C73CDDCE82E00E94C73CFA
:107D2000D9CE0E94763C809309020E94763C8093D3
:107D300008028091060190910701880F991F909386
:107D40000701809306010E94763C853409F4A6C0A1
:107D500080910C028E7F80930C020E94763C8032D0
:107D600009F0B8CE8091C00085FFFCCFF092C6002C
:107D7000609108027091090261157105B9F140E046
:107D800050E080910C02A82FA170B82FB27011C0E2
:107D9000BB2309F45CC0E0910601F0910701319624
:107DA000F0930701E09306014F5F5F4F46175707B7
:107DB000E8F4AA2369F3F999FECF209106013091E6
:107DC000070132BD21BDF89A90B58091C00085FFB2
:107DD000FCCF9093C6002F5F3F4F30930701209355
:107DE00006014F5F5F4F4617570718F38091C00099
:107DF00085FDE5CE8091C00085FFF8CFE0CE81E023
:107E00000E94C73C67CE0E94763C803209F08CCE3F
:107E10008091C00085FFFCCFF092C6008091C00029
:107E200085FFFCCFE092C6008091C00085FFFCCFAB
:107E3000D092C6008091C00085FFFCCFC092C600E2
:107E40008091C00085FFFCCFB092C60043CEE09188
:107E50000601F091070194918091C00085FFFCCF4D
:107E60009093C6009CCF80E10E94C73C33CE0E9415
:107E7000763C0E94763C182F0E94763C112309F430
:107E800083C0113009F484C08FE00E94C73C22CE29
:107E900080910C02816080930C02E5CE80910C02EF
:107EA000816080930C0259CF809107018823880F4D
:107EB000880B8A2180930B02809106019091070123
:107EC000880F991F90930701809306018091080203
:107ED00080FF09C080910802909109020196909359
:107EE000090280930802F894F999FECF1127E091D6
:107EF0000601F0910701C8E0D1E08091080290915D
:107F00000902103091F40091570001700130D9F34B
:107F100003E000935700E89500915700017001308D
:107F2000D9F301E100935700E89509901990009169
:107F3000570001700130D9F301E000935700E89534
:107F40001395103498F011270091570001700130FB
:107F5000D9F305E000935700E895009157000170B0
:107F60000130D9F301E100935700E895329602976A
:107F700009F0C7CF103011F00296E5CF112480919F
:107F8000C00085FFB9CEBCCE8EE10E94C73CA2CD19
:0C7F900085E90E94C73C9ECDF894FFCF0D
:027F9C00800063
:040000030000780081
:00000001FF
